:020000040000FA
:0400000009303A2861
:08000800A000030EA100831209
:1000100005191028831601178312B23081002B288E
:1000200083160113831203140B190310A80DA90DD5
:10003000AA0DAB0DAC0DAC16FF302C02031D2B2806
:10004000FA302B02031D2B2831152A08AF0029088E
:10005000AE002808AD008B100B11210E8300A00EFE
:04006000200E090065
:0C007400203084008001840A6030040207
:10008000031C3C281230B00063218316FF2390002C
:10009000831283160C308505870183128501870141
:1000A000073099000030831691009F008312C830FA
:1000B00083168100831231309000003083168C004B
:1000C000831210308B00831600309B001C141A081A
:1000D0008312BC00831610309B001C141A08831274
:1000E000BD00832181018E018F010B118B100B103C
:1000F0008C018B17892031198C20B30B87280310B2
:1001000085190314B90DF03039020319F6208C213A
:100110007A2864003210080031110130B7008B13C7
:100120002030370783169B001C141A088312A40082
:100130001030370783169B001C141A088312A30083
:10014000A6000230A6060030370783169B001C1459
:100150001A088312A200A7000130A7068B17321CD1
:10016000B72822090339A200A309A409A509240874
:100170002F02031DF02823082E02031DD528220874
:100180002D02031DF02801303702031DCC283D1835
:10019000CC283D143E14662102303702031DD528B9
:1001A000BD18D528BD143E14712126082E02031D4A
:1001B000F02827082D02031DF02801303702031D07
:1001C000E6283D1CE6283D103E147421023037021B
:1001D000031DEF28BD1CEF28BD103E147621F0282A
:1001E000B70A03303702031808008F280130B60021
:1001F000B300B400B500B70085018701B1138920B1
:10020000B30B1629031085190314B90DF030390208
:1002100003193D29B40B162901303702031979213E
:100220000230370203197D219630B400311DFF28BA
:100230003111321C20292D090339AD00AE09AF0957
:100240002F1CFF288E018F010C1CFF280C102E1E66
:10025000FF288B1320303707BB002F08BA0050212E
:1002600010303707BB002E08BA0050210030370786
:10027000BB002D08BA0050218B1785018701B70AF2
:10028000B60103303702031CFF28832108003E1CFF
:1002900008003E101030BB003D08BA005021080095
:1002A0008B133A0883161C159A003B089B005530A7
:1002B0009D00AA309D009C1464009C185C291C11B0
:1002C00083128B170800FF30C300080041101E3056
:1002D0004005031D0800C014C01A0800FF30C30009
:1002E0000800851285140800411408008516851041
:1002F00008000508113A850008000508223A850023
:10030000080008000800C001C1013D18C014BD1854
:100310008514BD1C851608008F08031908008F017D
:10032000C30F9A29C30A0310C00D41189A29C01A95
:10033000C015C012FC22C20068304005031D051024
:10034000401334304005031D051242080E02031805
:10035000B12914304005031D051408304005031D64
:1003600005168F08031D0800640042080E02031CD6
:10037000B12914304005031D051028304005031D28
:1003800005142C304005031D051210304005031DD7
:0E039000051601304302031D08004721080036
:0805F80003308A00430382076F
:100600000034043407340B340F34123416341934E4
:100610001C3420342334263429342C342F343334FE
:10062000363438343B343E3441344434473449342E
:100630004C344F3451345434563459345B345E3472
:10064000603462346534673469346C346E347034C9
:1006500072347434763478347A347C347E34803432
:10066000823484348634883489348B348D348F34A6
:100670009034923494349534973498349A349B342B
:100680009D349E34A034A134A334A434A634A734BA
:10069000A834AA34AB34AC34AE34AF34B034B13453
:1006A000B234B434B534B634B734B834B934BA34F7
:1006B000BB34BD34BE34BF34C034C134C234C3349F
:1006C000C434C434C534C634C734C834C934CA3455
:1006D000CB34CC34CC34CD34CE34CF34D034D0340D
:1006E000D134D234D334D334D434D534D534D634CD
:1006F000D734D734D834D934D934DA34DB34DB3492
:10070000DC34DD34DD34DE34DE34DF34DF34E03459
:10071000E034E134E234E234E334E334E434E43426
:10072000E534E534E534E634E634E734E734E834F8
:10073000E834E934E934E934EA34EA34EB34EB34CC
:10074000EB34EC34EC34EC34ED34ED34EE34EE34A4
:10075000EE34EF34EF34EF34F034F034F034F0347E
:10076000F134F134F134F234F234F234F334F3345A
:10077000F334F334F434F434F434F434F534F53439
:10078000F534F534F634F634F634F634F734F73419
:10079000F734F734F734F834F834F834F834F834FC
:1007A000F934F934F934F934F934FA34FA34FA34DE
:1007B000FA34FA34FA34FB34FB34FB34FB34FB34C4
:1007C000FB34FB34FC34FC34FC34FC34FC34FC34AB
:1007D000FC34FD34FD34FD34FD34FD34FD34FD3492
:1007E000FE34FE34FE34FE34FE34FE34FE34FE3479
:0E07F000FE34FF34FF34FF34FF34FF34FF3497
:084000000B000300040008009E
:02400E00CC01E3
:10420000010078007A007C007E007B0079007F004E
:104210007D007A0078007E007C00FF00FF00FF0038
:104220000000F200F600FA00FE00F200F600FA00CC
:10423000FE00F200F600FA00FE00FF00FF00FF00A3
:10424000010005000500050005000900090009003E
:1042500009000D000D000D000D00FF00FF00FF0024
:10426000FF00FF00FF00FF00FF00FF00FF00FF0056
:10427000FF00FF00FF00FF00FF00FF00FF00FF0046
:10428000FF00FF00FF00FF00FF00FF00FF00FF0036
:10429000FF00FF00FF00FF00FF00FF00FF00FF0026
:1042A000FF00FF00FF00FF00FF00FF00FF00FF0016
:1042B000FF00FF00FF00FF00FF00FF00FF00FF0006
:1042C000FF00FF00FF00FF00FF00FF00FF00FF00F6
:1042D000FF00FF00FF00FF00FF00FF00FF00FF00E6
:1042E000FF00FF00FF00FF00FF00FF00FF00FF00D6
:1042F000FF00FF00FF00FF00FF00FF00FF00DD00E8
:00000001FF
